:0A00000030C0FECFFDCFFCCFFBCFD8
:10000A00FACF46C0F8CFF7CFF6CFF5CFF4CFF3CF7C
:10001A00F2CFF1CFF0CFEFCFEECFEDCF0300020258
:10002A0001030302030303010300030300030000A7
:10003A00E424E1652545C524E565A5C5C0E5C1817A
:10004A0001210000FCF3CF006400C80090012003E6
:10005A00F8FFFCFFFEFFFFFFF894EE27ECBBE5BFBD
:10006A00F8E1A4B7A77FA4BFF1BDE1BD8DE0A2E08E
:10007A00ED938A95E9F780E8A0E6ED938A95E9F78A
:10008A00E0E0E3BBE4BBE5BBEFEDEDBFC0E88FC04A
:10009A000A92AA93EA93FA93EFB7EA93E2B3EF6369
:1000AA00E2BB85D1EA5DFF4F04900BBA80D1E65CD2
:1000BA00FF4F049008BA989B03C0E1E0E31509F0EA
:1000CA0001C0C49AE2B3AE2FE32D76D1E25BFF4FB3
:1000DA00E491EA23E2BB3394E2E0E31508F4332423
:1000EA00E991EFBFF991E991A9910990189524979F
:1000FA00B1D2A20100244014500414F0E2E106C077
:10010A00FA01E095F0953196AF01E0E1E0938900BC
:10011A00989AFA0172D2E887F987FA01EF70F070BB
:10012A00EE83FF83AAE0B0E081D267D20E2F188552
:10013A00143658F0E12F40D1E456F040EA932ED11C
:10014A003E2FE1E0E093890003C01A9327D13E2FA6
:10015A00143638F4A0918900A03111F41A3008F449
:10016A0008C098982BD1E0938A00E32FEF70E093B0
:10017A008B00A0918900A03111F41A3008F004C054
:10018A00EAE81083EBE80083A0918900A23111F418
:10019A00143608F009C012D1309719F00FD1E09344
:1001AA008900E32FEF700ED15CD22A960895E0E021
:1001BA00EBBBE3E0EABBE0E0E8BBEFEFE7BBEFE372
:1001CA00E2BBEFEFE1BBE0E0E0BFE3E0E3BFE0E08A
:1001DA00E2BFE6BFECBFEFBDEEBDEDBDECBDE5BDD8
:1001EA00E4BDEBBDEABDE9BDE8BDEBBFE5BFE2E0BA
:1001FA00E9BFE0E0EDB9E0E8E8B911D1E0EFEA9350
:10020A00ECE8EA935CD10E2F7894EFE0E093890052
:10021A00E2E1D8D0013088F010E0101768F4D7D0A6
:10022A00A081A03121F4D3D0EA9368D02F01E8EE5F
:10023A00F3E0D2D01F5FF1CF03C0E0EDF7E0CCD0FE
:10024A000130E8F010E01017D0F4C1D0A081A83234
:10025A0021F4BDD0EA9372D02F01B9D0A081A03188
:10026A0021F4B5D0EA934AD02F01B9D0E415F505A7
:10027A0009F03DDFE0EDF7E0AFD01F5FE4CFE0CF5C
:10028A00FFCF1A93CCD0E03011F4E0E084C0E981CA
:10029A00E03079F0F894E5E5A5D0789410E0F89488
:1002AA00A981ED91A9839ED078941F5F1830B8F385
:1002BA0004C0F894ECEC96D07894E1E06CC0CED10E
:1002CA00EA8192D011F4E0E016C0F894EEEB8AD0FD
:1002DA00789410E000E8F8940F930F5FE1D0AF91A3
:1002EA00EC9378941F5F1930B0F3E0E8EA93E9E001
:1002FA00EA9354D18BD1B9D123960895E88174D069
:10030A0011F46DD019C0F894E4E46CD07894E6E264
:10031A00F2E062D0E8816CD011F461D00DC0F8949B
:10032A007ED07894F0918100E0E0DF01E0918000D6
:10033A0043D0EA2BFB2B51D1219608951A93E981D8
:10034A0057D011F44CD027C0A0918400B0E0E5E06A
:10035A003BD1E3701E2FE98147D011F440D01BC076
:10036A00F894E4E43FD07894E12FA2E5B0E044D0D9
:10037A0033D0E9813DD011F432D00DC0F8944FD07A
:10038A007894E12FAAE5B0E037D0A0918000B0912F
:10039A008100EA23FB23188122960895A991EE276A
:1003AA00AA5012F0E05FFCCFA65FEA0F0895A9E811
:1003BA00A30DEC91F0E00895F0E00895E32FFCDF3F
:1003CA0013D10895E0938A00EBE800830895E12FA2
:1003DA00A9E021D1E4570895FA93EA9314C0E1EF12
:1003EA00F8ED0895EA9361C0EA934BDFE03008958F
:1003FA00EA9365DFE0300895DFDFEE0FFF1FEA0FB3
:10040A00FB1F24D10895E991F991309639F088EECD
:10041A0093E00197F1F7A8953197C9F70895EE2768
:10042A0096988E9A80EE91E00197F1F78E9883E183
:10043A008A95F1F7869B089585E68A95F1F7869B5A
:10044A00E39586E891E00197F1F708958E9A83E0A3
:10045A008A95F1F78E988FE08A95F1F788948699B4
:10046A000894E7958BE68A95F1F70895E8948E9AB1
:10047A0083E08A95F1F770FD8E9881E18A95F1F70C
:10048A00869903C070FF03C0089570FF089584E63B
:10049A008A95F1F78E9887E08A95F1F7689408951E
:1004AA0068E0D4DF6A95E9F7089568E07991EE2764
:1004BA00DDDF26F477956A95D9F7E39508954F938A
:1004CA005F9311244427A881BB27012C1124A7DF9D
:1004DA00EE23F9F0E981EA93E8DF51E0501598F448
:1004EA00B5DFE7FD08C0B2DFE7FD06C03FD08923CC
:1004FA0019F4152E01C0AADF39D0892370E009F05A
:10050A0071E0B4DF1EC0A2DFE7FF0BC09FDFE7FF89
:10051A0005C0E42F5F914F9122960895689436D0D2
:10052A00EFCF94DFE7FF01C003C0501531F0152E5D
:10053A00E8942CD077279ADF04C0689427D071E01A
:10054A0095DF5395513454F281DFEE1FEE1FE170AF
:10055A001896EC93189743951120D9F259E0EC912B
:10056A001996EC9318975A95D1F7AFCFE52FEA95DC
:10057A006E2FE695E695E695EA0FFF27808191E0D2
:10058A00677019F0990F6A95FCCF0895EFDF1EF096
:10059A009095892301C0892B80830895EE2788814D
:1005AA00882381F068E1A981BB2798E0FD917F2F1C
:1005BA007E27779508F4E627E795F6959A95B9F791
:1005CA008A9599F722960895EE230E2EFD0121F0C1
:1005DA00F595E7950A94E1F70895EE0FFF1FEE0FE0
:1005EA00FF1FEE0FFF1F0895F595E795F595E7951F
:1005FA00F595E795F595E7950895F695E795F695B6
:10060A00E795F695E795F695E7950895EE23E1E0E7
:10061A0009F0EE2708950A2EAA1BB9E003C008F4D0
:10062A00A00DA695E795BA95D1F708950A2E1B2E27
:10063A0081E1AA27BB1B05C010F4A00DB11DB69518
:10064A00A795F795E7958A95B9F708950590F491D6
:10065A00E02D08955A934A933A932A931A930A9348
:10066A0008955D814C813B812A8119810881089511
:00000001FF
